:10000000A52B820700340034013401340234023459
:100010000334033404340534063407340834093413
:100020000A340B340C340E341034123414340F30C0
:10003000831201058207000000000000000000009C
:1000400000000000000000000000000000000000B0
:100050000000000045088500E2308100410884006E
:100060000508C200C30A0008C400840A0008C500CD
:10007000840A4C30841E0408C1004408850008002E
:10008000A2011430220203184B284C3022078400AE
:100090008001A20A41284C30C100C501FC3081001A
:1000A000172883160F170F1F8F120F1B8F168F1E07
:1000B0000F128F1A0F16FF27900008308500831249
:1000C00010100C1008308316810083121016901641
:1000D000101419159914191483169F0183128501A0
:1000E0000800A3000E08B60033083602031CB40A49
:1000F0003608B30023083607B5000E083506031D81
:100100007D280800A200B401C830340203189028EA
:100110002230850022087120850122087120842860
:100120000800B401C8303402031899280A3071203D
:1001300092280800B301B4018E01AE308220CF3086
:100140008220912091209120CF308220C3308220C4
:10015000AE3082206730822091206730822091204B
:10016000823082209120912091288312A3008C1349
:10017000220883169B008312230883169A001C15FD
:1001800055309D00AA309D009C141C1183128C1FB9
:10019000C62883128C138312031308008312A20053
:1001A000220883169B001C141A088312A3008312D2
:1001B0000313230808000030CE20B90039082A3A7A
:1001C000031DE6280130CE20B900EA28A2012A301A
:1001D000B520B90108001C30BA001C30BB001C302F
:1001E000BC001C30BD004E30BE004E30BF004E3053
:1001F000C0000800BA1B17281720AD0803190229F0
:100200001C30BA00BA031720BA1F0F290130A20010
:100210003908B52017200A30AB000A30AC00BB1BF0
:100220002D291720AC1F1829ED302C02031C1A2988
:100230001C30BB001720AB1B212914302B020318E4
:100240002A291720AB1F2829ED302B02031C2A294D
:100250001C30BB001720BB033F291720AB1B3729DD
:1002600014302B02031C3729391417203829391070
:1002700017201C30BB000A30AB000A30AC0017203E
:10028000BC1B5E291720AC1B492913302C02031814
:100290004B291C30BC001720AB1B522913302B02FA
:1002A00003185B291720AB1F5929EC302B02031CC4
:1002B0005B291C30BC001720BC036E291720AB1B28
:1002C000682913302B02031C6829B91417206929E7
:1002D000B91017201C30BC00AB01AC011720BD1BAE
:1002E0007D291720AD1B782928302D0203187A2983
:1002F0001C30BD001720BD038A2917202B08BE071C
:100300002C08BF072E08C0071C30BD000A30AB0008
:100310000A30AC001720AD0117281720C601C30111
:1003200017200830050529060319C729C31F90297E
:10033000C30117200830050529060319C729C31F63
:100340009929C30117200830050529060319C72973
:10035000C31FA229C3011720083005052906031968
:10036000C729C31FAB29C30117200830050529067B
:100370000319C729C31FB429C30117200830050575
:1003800029060319C729C31FBD2917200134C3013A
:1003900017200830420529060319C60A1720003421
:1003A0001720A301043023020318102A1720343029
:1003B000C3021720083005052906031DE329C31BC6
:1003C000D92917200134172034304307B7001720EC
:1003D000B71BED2905303702031C0134C930C307B0
:1003E00017200830050529060319FA29C31BF0292F
:1003F0001720013417206A304307B70017202B302D
:1004000023078400370880000230C3001720B71B81
:100410000C2A32303702031C01341720A30AD229D8
:1004200017202A08033A031D1E2A2D08B70017209B
:100430002E08AD003708AE001720003417202A0B15
:100440002A2A2C08B70017202D08AC003708AD0069
:10045000172000341720AA08031D3C2A2B08B700D8
:1004600017202C08AB003708AC002C08B700172069
:100470002D08AC003708AD001720003417202F08D6
:100480002B07AF000310AF0C2F08AB00172030086C
:100490002C07B0000310B00C3008AC001720310856
:1004A0002D07B1000310B10C3108AD001720320840
:1004B0002E07B2000310B20C3208AE0017203E081F
:1004C000AB023F08AC023C30AD024008AE02172040
:1004D000AD1BAD01FA201720391C742A2B08B70078
:1004E0002C08AB023708AC071720AB1F7C2AAB09DE
:1004F000AB0A0130B3007E2A0230B3001720AC1FD4
:10050000862AAC09AC0A1030B400882A2030B40026
:100510001720AE1F8F2AAE09AE0AB601902AB60187
:1005200017200314AD1F0314AD1F0310AD0C1720CB
:10053000AB1BA02A15302B02031CA02A1430AB00E1
:100540001720AC1BA92A15302C02031CA92A143031
:10055000AC001720AD1BB22A15302D02031CB22AA5
:100560001430AD001720AE1BBB2A15302E02031C21
:10057000BB2A1430AE001720B91C172817202B08EF
:100580000120AB0017202C080120AC0017202E08FA
:100590000120AE001728A501A601A701A801172078
:1005A000A30114302302031817281720A2012B08D7
:1005B000A502A51FE02A17201430A5073308A207BB
:1005C00017202C08A602A61FEA2A17201430A60717
:1005D0003408A20717202D08A702A71FF42A172006
:1005E0001430A7073508A20717202E08A802A81F55
:1005F000FE2A17201430A8073608A20717204C300F
:1006000023078400220880001720A30AD12AAD0105
:10061000B8010430B500080017200C30C700803046
:100620000F07C8000800172048080F028039031D73
:10063000172817208030C807C708031D482B17202C
:100640000C30C7000430AB000130B3001720391C58
:100650002C2B0430AC002D2BAC0117201030B40033
:100660003808AD000430AE00B6011720CB221720A9
:100670000314AD1F03102D0CB7002D08B70717206A
:100680000314B71F0310370CAD0017202D08B80056
:10069000C703172817200C300F07CA0004300F07B4
:1006A000C900172049080F02803903196E2B172043
:1006B000083005052906031D6C2B172004300F0791
:1006C000C9002908083CA90017204A080F028039F0
:1006D000031D6C2B172001341720522B17200034D8
:1006E00017200230AA0017204A23003A03197A2B58
:1006F0001720742B8D21003A031D732B1720D02156
:10070000003A0319852B1720732BB3011720A20180
:10071000043022020318172817202B3022078400E8
:100720000008B70017204E30B702B71F992BB70942
:10073000B70A172033083702031CA22B3708B3006F
:100740002208AA001720A20A882B51209A20DB2019
:100750000723A001EB20A901A10104302102031805
:10076000B82B2F30210784004E308000A10AAD2B1A
:1007700040207023A00803190C2317200430A00088
:1007800017201720A008031D132317204A23003A1F
:10079000031DE32B17208D21003A031DE32B1720A7
:1007A000D021003A031DE32B17203E221720A0087A
:1007B0000319DD2BA0031720C12B1720CB221720F4
:0A07C0002D08B800C12B1720BA2B3A
:020FFE000034BD
:044200002A00000090
:02400E00C433B9
:00000001FF
